:100000000C9479040C94B1040C94B1040C94B104D4
:100010000C94B1040C94B1040C94B1040C94B1048C
:100020000C94B1040C94B1040C9473260C942F26F8
:100030000C94C6270C94B1040C94B1040C94B10434
:100040000C94B1040C94B1040C94B1040C94B1045C
:100050000C94B1040C94A2270C94B1040C94B10438
:100060000C94B1040C94B1040C94B1040C94B1043C
:100070000C94B1040C94B1040C94B1040C94B1042C
:100080000C94ED270C94B1040C94B1040C94B104BD
:100090000C94B1040C94B1040C94B1040C94B1040C
:1000A0000C94B1040C94B1040C94B104076342366F
:1000B000B79BD8A71A39685618AEBAAB558C1D3CF9
:1000C000B7CC5763BD6DEDFD753EF6177231BF00BD
:1000D0000000803F08000000BE922449123EABAAF7
:1000E000AA2ABECDCCCC4C3E00000080BEABAAAA52
:1000F000AA3E00000000BF000000803F000000009A
:1001000000084178D3BB4387D1133D190E3CC3BDD2
:100110004282AD2B3E68EC8276BED98FE1A93E4C7F
:1001200080EFFFBE01C4FF7F3F00000000000631EA
:10013000FF0974A1010975150026FF0095207508B7
:1001400081020976150026FF00952075089102C0EE
:1001500005010980A101850319012AB700150126AF
:10016000B700950175108100C0050C0901A101853A
:100170000419012AA002150126A00295017510811B
:1001800000C005010906A101050719E029E71500CE
:100190002501950875018102950175088101050702
:1001A000190029FF150026FF009506750881000536
:1001B00008190129059505750191029501750391AD
:1001C00001C064796E616D6963206D6163726F3A1D
:1001D00020736C6F7420256420706C617962616398
:1001E0006B0A0064796E616D6963206D6163726F83
:1001F0003A20736C6F742025642073617665642CDB
:10020000206C656E6774683A2025640A0064796E14
:10021000616D6963206D6163726F3A207472696DFC
:100220006D696E67206120747261696C696E672008
:100230006B65792D646F776E206576656E740D0A37
:1002400000000000000000000000000000000000AE
:10025000000000000000000000000000000000009E
:1002600000000000007E0F00D4FFFFFFC700000069
:100270007800000000000000002A2B280000000089
:100280000000000000000000000000002900000045
:10029000002C1E3420212224342627252E362D37EB
:1002A00038271E1F202122232425263333362E37BC
:1002B000381F0405060708090A0B0C0D0E0F101154
:1002C00012131415161718191A1B1C1D2F31302361
:1002D0002D350405060708090A0B0C0D0E0F101129
:1002E00012131415161718191A1B1C1D2F3130352F
:1002F0004C64796E616D6963206D6163726F3A2041
:1003000069676E6F72696E67206D6163726F2070CE
:100310006C6179206B6579207768696C65207265FE
:10032000636F7264696E670D0A006272616E646F5A
:100330006E28313229466562323032320068616E91
:100340006E6168283238294D6179004C65616E67AD
:100350002E486F756E40416476616E6365644269D4
:100360006F6E6963732E636F6D006C65616E676895
:100370006F756E40676D61696C2E636F6D006261B1
:10038000636B6C696768742064656372656173652B
:100390003A2025750A006261636B6C696768742096
:1003A000696E6372656173653A2025750A00626142
:1003B000636B6C6967687420737465703A20257587
:1003C0000A0044454255473A2064697361626C658E
:1003D000642E0A0044454255473A20656E61626CBE
:1003E00065642E0A0029001E001F00200021002243
:1003F00000230024002500260027002A002B0014DB
:10040000001A00090013000A000D000F0018001C5C
:100410000033003400A95D04001500160017000722
:10042000000B00110008000C0012002800E1001D64
:10043000001B000600190005000E001000360037F2
:100440000038005200E000AC5DE200E300AA5D2C41
:10045000002C00AB5DB15D50004F00510029001E23
:10046000001F002000210022002300240025002678
:100470000027002A002B0014001A0008001500179E
:10048000001C0018000C00120013003400A95D04C9
:10049000001600070009000A000B000D000E000FF7
:1004A0000033002800E1001D001B000600190005B4
:1004B00000110010003600370038005200E000AC98
:1004C0005DE200E300AA5D2C002C00AB5DB15D5045
:1004D000004F005100010001000100010001000176
:1004E000000100010001000100B25D4C00010001AB
:1004F00000010001000100010001004A0052004D0E
:10050000004B00210AA95D3A003B003C003D003E43
:10051000003F00500051004F004E0001000100401C
:100520000041004200430044004500010001000179
:1005300000010001000100AC5D01000100AA5D01A5
:10054000000100AB5D01000100010001000100019C
:100550000001000100010001000100010001000193
:1005600000540055000100010001000100010001DC
:1005700000010001005F00600061005600A95D01FC
:10058000000100010001000100010001005C005DAC
:10059000005E0057000100010001000100010001A0
:1005A000000100010059005A005B0001000100AC8D
:1005B0005D01000100AA5D01000100AB5D62000168
:1005C000006300580001000100010001000100016A
:1005D0000001000100010001000100010001000113
:1005E0000001000100010001000100010001000103
:1005F0000001003500A95D010001000100010001BA
:100600000001002D002E0001000100010001000189
:10061000000100010001000100010001002F003075
:1006200000310001000100AC5D01000100AA5D0184
:10063000000100AB5D01000100010001000100ADFF
:100640005DAE5DAF5DB05D0100010001000100071E
:100650005D085D065D01000100010001000100016F
:1006600000010001000100045D055D0100A95D01BC
:100670000001000100010001000100010001000172
:10068000000100A8000100010001000100010001BB
:100690000001000100010001000100A9000100ACFF
:1006A0005D01000100AA5D01000100AB5DAE00BC70
:1006B00000BB00AA000100A75DA85D0100010001C8
:1006C0000001000100010001000100005C010001C7
:1006D0000001000100010001000100010001000112
:1006E0000001000100A95D010001000100010001FD
:1006F00000010001000100010001000100010001F2
:1007000000010001000100010001000100010001E1
:1007100000010001000100AC5D01000100AA5D01C3
:10072000000100AB5DB35D0100010001004F6E658B
:1007300073686F743A206163746976653A20256442
:100740000A000A002530325820006B6579626F611B
:1007500072645F7265706F72743A20005B735D0043
:100760000A002530313662003A2000253032580028
:100770000A722F63203031323334353637383941FD
:1007800042434445460A000A0025303258006C6551
:10079000645F7461736B3A20006261636B6C6967BC
:1007A00068742064697361626C650A006261636BDE
:1007B0006C6967687420656E61626C650A006261CD
:1007C000636B6C6967687420746F67676C653A2047
:1007D00025750A005B435D005B445D005B535D0073
:1007E0005B575D005B525D0009025B00030100A0E6
:1007F000FA090400000103010100092111010001AF
:1008000022400007058103080001090401000103DB
:1008100000000009211101000122320007058203B6
:100820002000010904020002030000000921110157
:1008300000012222000705830320000107050303AE
:100840002000011201000200000008A803F3670263
:10085000000102000110035000720065006F006E7D
:10086000006900630000000A034F004C004B004287
:100870000000000403090464796E616D6963206DF2
:100880006163726F3A20736C6F74202564206C650D
:100890006E6774683A2025642F25640A0064796EB7
:1008A000616D6963206D6163726F3A2069676E6F75
:1008B00072696E672061206C656164696E67206B88
:1008C00065792D7570206576656E740D0A00647902
:1008D0006E616D6963206D6163726F207265636F15
:1008E0007264696E673A20737461727465640D0A8C
:1008F000000011241FBECFEFDAE0DEBFCDBF04B68B
:1009000003FE18C08091A9099091AA09A091AB0992
:10091000B091AC098730904BA740B04B59F410927E
:10092000A9091092AA091092AB091092AC09E0E053
:10093000F8E3099529E0A8E5B5E001C01D92A93AC0
:10094000B207E1F715E0A0E0B1E0E0E9F3E602C0AC
:1009500005900D92A835B107D9F70E949C290C94F7
:100960009A310C940000FF93EF93E0915805F091B9
:100970005905309709F00995EF91FF910895FC0111
:100980008591803011F0EFDFFBCF0895FF27E0E283
:1009900030E247FF0CC0419597FF09C0EDE260953A
:1009A000709580959095611D711D811D911D27FF8A
:1009B00002C0219530E350E2AA27660F771F881FF7
:1009C000991FAA1FA41710F0A41B63955A95A9F7A5
:1009D000AA3008F0A95FA05DAF93F395611571058A
:1009E0008105910541F7ED3211F4EF93F395F2177C
:1009F00018F43F93F395FBCF8F91B5DFFA95E1F7AC
:100A00000895E991F9918591803021F0853219F0AE
:100A1000AADFF9CF089520E0E89455915532C1F34B
:100A2000503311F4689455915A3348F4505390F36D
:100A3000220F022E220F220F200D250FF4CF0EF4CD
:100A4000219589919991533619F3533729F15335EB
:100A500059F1BC0188279927E8945C3621F48991E3
:100A6000999168945591543639F446EF7EF077FFAA
:100A70000DC08FEF9FEF0AC055374AE039F0583567
:100A800040E121F0523642E009F00895FF93EF93E0
:100A90007DDFEF91FF91B7CFFF93EF93FC01819141
:100AA0008030B9F360DFFBCFFF93EF9368DFF1CFC6
:100AB000DF93CF93CDB7DEB72596A3DFCF91DF913C
:100AC0000895E8EDF0E080818E7F80831092E2004F
:100AD0001092DA001092E100A0EEB0E08C918160FB
:100AE0008C9380818F77808319BCA7EDB0E08C91C7
:100AF0008E7F8C9380818F7E80831092320908953F
:100B00002091E4003091E50095E6A9012091EC00E8
:100B1000822F817020FF06C08091E80080FF06C010
:100B200080E008952091E80022FD1AC080913F09DD
:100B3000882389F0853089F08091EB0085FD0FC016
:100B40002091E4003091E50042175307F9F29150EB
:100B5000E1F684E0089582E0089583E0089581E05D
:100B60000895EF92FF920F931F93CF937C018B0117
:100B70000E948005C82F811117C08091E80085FD73
:100B80000BC08091E8008E778093E8000E9480057A
:100B9000882399F3C82F08C0F70181917F018093C2
:100BA000F1000150110949F78C2FCF911F910F913E
:100BB000FF90EF9008958091410987FF13C08091C5
:100BC000E80082FF06C08091E8008B778093E80000
:100BD00004C080913F098111F2CF089580913F09AF
:100BE0008823D9F38091E80080FFF8CF8091E80056
:100BF0008E77ECCF982F9093E900242F762F50E03A
:100C0000891731F07091EC002091ED005091F000C7
:100C100021FD07C09F5F973071F78093E90081E065
:100C200008953091EB003E7F3093EB003091ED0062
:100C30003D7F3093ED003091EB0031603093EB005D
:100C40007093EC002093ED005093F0002091EE00A3
:100C500027FDE0CF80E00895CF92DF92EF92FF92E0
:100C60000F931F93CF93DF93C8EDD0E088818F7EE1
:100C70008883E7EDF0E080818160808384E082BF3B
:100C800081E08093320988818E7F888302EE10E0B4
:100C9000F80110821092DA0081EEC82ED12CF601F4
:100CA000108288818F778883888180688883888193
:100CB0008F7D888319BC10923F09109240091092D1
:100CC0003E0910923D0990EEE92EF12CF70180814A
:100CD0008B7F808388818160888342E060E080E050
:100CE0000E94FA05F60180818E7F8083F801808161
:100CF00081608083808188608083F70180818E7F1E
:100D00008083888180618883DF91CF911F910F91CB
:100D1000FF90EF90DF90CF900895FC0180914709FC
:100D20009091480986179707A0F06115710529F47D
:100D30009091E8009E779093E80090E0611571052E
:100D400051F4911108C08091E80082FF34C080E026
:100D50000895BC01F2CF80913F098823C1F185300D
:100D6000C1F18091E80083FD30C08091E80082FDF0
:100D7000EACF8091E80080FFE1CF8091F3002091DD
:100D8000F200382F6115710519F02830310558F03F
:100D900091E02830310509F090E02091E8002E77AD
:100DA0002093E800CBCF81918093F10061507109CD
:100DB0002F5F3F4FE7CF80913F09882341F0853077
:100DC00041F08091E80083FFBECF81E0089582E08A
:100DD000089583E008950895089580913409089551
:100DE0009C014FB7F8948091280990912909A0910E
:100DF0002A09B0912B094FBF821B930B08952FB77F
:100E0000F8948091280990912909A0912A09B0911C
:100E10002B092FBF08952091250930912609281705
:100E2000390771F09093260980932509E0912309F1
:100E3000F0912409309721F00084F185E02D099488
:100E4000089520912109309122092817390771F05E
:100E50009093220980932109E0912309F0912409BC
:100E6000309721F00680F781E02D09940895E091F4
:100E70002309F0912409309721F00190F081E02DB1
:100E8000099480E008958F929F92AF92BF92EF9263
:100E9000FF920F931F93CF93DF938430B8F58111A6
:100EA00036C090918000977F909380002F98A091FA
:100EB0008600B0918700282F30E00E94792D23E032
:100EC00030E040E050E00E94572D89019A01809166
:100ED0008600909187006CE070E00E944C2C6017B7
:100EE0007107D8F0C80169E070E00E944C2C709343
:100EF0008D0060938C00DF91CF911F910F91FF9037
:100F0000EF90BF90AF909F908F90089583E0909165
:100F10008000986090938000CACF80918600909165
:100F20008700E0908600F0908700E0918600F091C5
:100F30008700C6E0D0E0BE010E944C2C060F171FB0
:100F4000211D311D4801590185E0880C991CAA1CFE
:100F5000BB1C8A95D1F7C701BE010E944C2C9F0192
:100F600050E040E0260F371F411D511DC501B4015F
:100F70000E94572D49015A01E0918600F0918700A7
:100F8000CA01B9010E94302C9B01AC01DF010E9413
:100F9000442D9B01AC01C501B4010E94302C2FE00F
:100FA00096958795779567952A95D1F70091860054
:100FB0001091870030E020E006171707280739074F
:100FC00008F095CF609186007091870090CFE1E79F
:100FD000F0E080818D7F8083E0E9F0E080818F7395
:100FE00080830895CF92DF92EF92FF926B017C0194
:100FF00020E030E0A9010E94F52D81110AC0809106
:1010000090008F7380939000FF90EF90DF90CF90CF
:10101000089580919000806880939000C092160996
:10102000D0921709E0921809F092190920E030E0F7
:1010300040E051E4C701B6010E94B62F9B01AC010C
:1010400060E074E284E79BE40E94FA2D6B017C016E
:101050000E94732E709397006093960060919204A3
:1010600070E090E080E00E94A42EA70196010E940B
:10107000B62F20E030E048EC52E40E94FA2D0E94A6
:10108000732E7093990060939800BECF8091D00327
:10109000811122C01092A5090E94E70710925C09F5
:1010A00010925D091092510910925009E5E6F9E09D
:1010B00080E090E0A0E8BFEB1182108282839383EE
:1010C000A483B58317821682389629E0E53AF207A1
:1010D00099F781E08093D003089580911E098111D2
:1010E0000C9446080895F894E82FE295EF70F0E02C
:1010F00031A1282F2F7081E090E001C0880F2A9540
:10110000EAF7982F9095932391A392A1892B82A31C
:10111000789408959091E60892FF06C0282F2871D0
:101120002830F9F4877F846093FF06C0282F287148
:101130002831F1F4877E84612091E70820FF06C002
:10114000382F38713830D9F4877F816021FF06C08D
:10115000282F28712831D1F4877E816194FD877E04
:101160000895282F24712430F9F68B7F8860DCCF16
:10117000282F2471243101F78B7E8861DDCF382F31
:101180003171313019F78E7F8860E0CF282F2171BF
:10119000213121F78E7E8861E1CFCF93DF93EC017F
:1011A00082389105A9F1D8F58133910509F496C0EB
:1011B00048F58932910509F48AC08A9709F495C0E7
:1011C000C11522E5D20708F0B6C0C11531E5D30735
:1011D00008F026C1C83ED10508F09CC0C03ED1052C
:1011E00060F5C83AD10508F087C0C53AD10508F0C6
:1011F000EFC0C130D10509F12097F9F0C430D10515
:10120000E0F440C08533910509F45AC0C997C1F68E
:101210008091E608837089F0C0EED0E00EC0833E76
:10122000910599F170F4803E910501F1823E91059E
:1012300039F68091E60882FD21C0CE01DF91CF9181
:101240000895863E910561F1873E910571F1843ED6
:10125000910509F0B5CF8091E70881FFEECF80912D
:10126000E608C7EED0E084FD0DC0E7CF8091E60828
:1012700080FD07C19091E70890FFDFCFC3EED0E07B
:1012800084FFDBCFD0E0C0E0D8CF8091E60882FDBC
:10129000FBC09091E70890FDBFCF84FFCECFF2CF87
:1012A0008091E60883FDDDCFC8CF8091E60883FDFD
:1012B000EEC09091E70891FFF0CFC4EED0E0BDCF33
:1012C0008091E60885FFB9CFC9E2D0E0B6CF809122
:1012D000E60885FFB2CFC5E3D0E0AFCF8091E60846
:1012E00086FFABCFCAE2D0E0A8CF8091E60886FFA8
:1012F000A4CFC1E3D0E0A1CFCF3BD10518F6C85AA7
:10130000D0E0CC0FDD1FC754DB4F0990D881C02D32
:10131000D46493CFC11540E5D40708F064C0C1156B
:1013200080E4D80708F05CC0CE019A9581159F41F2
:1013300008F483CFA7CFC11536E5D30718F5C1153B
:1013400045E5D40708F084C0C11584E5D80708F046
:101350007AC09C2F969596959E0123703327C115D0
:10136000D34508F462C0C1E0D0E002C0CC0FDD1F5D
:101370002A95E2F730E2939FC0011124C82BD92BA4
:10138000DA685BCFC1158AE5D80778F4C11599E50D
:10139000D90708F068C0C11528E5D20708F472CF54
:1013A000DC2FCC27C06FD06A48CFCE019056811574
:1013B000904208F067CF8D2F8F710E948A0890E0CD
:1013C000982F882788279F719C012C2BE90149C001
:1013D000C55AD0E0CA54DB4FC881D0E0D0642DCFCD
:1013E000DF70D06A2ACFCE01E4E096958795EA9522
:1013F000E1F783702C2F26952695237040E2249FD9
:1014000090011124382B8C2F8370C1E0D0E002C0F2
:10141000CC0FDD1F8A95E2F7C22BD32BDC680DCFF2
:10142000DC2FCC27C16FD06A08CFC1E0D0E002C06A
:10143000CC0FDD1F2A95E2F720E2929FC001112414
:10144000C82BD92BEBCFDC2FCC27C46FD06AF5CEBD
:101450008C2F0E948A08C82FD0E0DC2FCC27CC2705
:10146000DF71D062EACE8C2F8F700E948A0834E040
:10147000D695C7953A95E1F7CF709C2FEC01D069CE
:10148000DCCEC9E3D0E0D9CEC2EED0E0D6CEC6EEF7
:10149000D0E0D3CE8091D10881111092D108089567
:1014A00080959091D00898239093D0080895ECE50A
:1014B000F5E09191891303C0DF0111971C9295E02B
:1014C000E236F907B1F70895ACE5B5E0EFEF90E04B
:1014D0002D91821751F0EF3F19F4211101C0E92F2E
:1014E0009F5F9630A9F7EF3F09F408950E2E000C88
:1014F000FF0BE65AFA4F828308958091C5089091B8
:101500009408981301C008958F5F8770FACFAF9247
:10151000BF92CF92DF92EF92FF920F931F93CF93E0
:10152000DF93C0904909D0904A09E0904B09F090B0
:101530004C094091D2085091D3086091D408709121
:10154000D508C42AD52AE62AF72ACFE1D0E0082F09
:1015500010E02CE0929F000D111D11249CE3A92E98
:10156000BC2ED701C6010C2E04C0B695A795979541
:1015700087950A94D2F780FD0FC0219788F7B12C88
:101580008B2DDF91CF911F910F91FF90EF90DF9006
:10159000CF90BF90AF900895AC9EF001AD9EF00D3E
:1015A0001124E00FF11FEE0FFF1FEB51FC4F85914F
:1015B00094910E94CD08019701F3E2CFCF93DF937E
:1015C000EC010E94870AEC2FF0E09CE0D99FE00D2F
:1015D000F11D11249CE3899FE00DF11D1124EE0FF4
:1015E000FF1FEB51FC4F85919491DF91CF910C94AB
:1015F000CD082CE0929F800D1124982F977086952E
:101600008695869525E0829FF0011124EA59F74FCF
:1016100050E040E080E0219130E0092E02C0369594
:1016200027950A94E2F721703327042E01C0220F78
:101630000A94EAF7822B4F5F5F4F4530510559F707
:1016400008952CE0929F800D1124982F977041E00F
:1016500001C0440F9A95EAF786958695869595E0A0
:10166000899FF0011124EA59F74F90E080E070E083
:101670005191DF0111979B01082E02C036952795E5
:101680000A94E2F7217021952527242325272C93FE
:1016900001968530910561F70895FC018081918163
:1016A0000E94DE0A92959F70963091F058F4925FF6
:1016B0009F70923058F4803F19F030F4883E30F437
:1016C00081E008959A5FF4CF843FD1F380E00895DC
:1016D000883EB0F3813FD1F7F3CF829590E09C0133
:1016E000220F331F220F331F2C7C959587959595DC
:1016F00087958373282B30E0C901880F991F8A7A58
:10170000359527952575822B08959FB7F8941092EB
:1017100030099FBF90913F09943009F048C0209153
:10172000E9002F703091EC00932F917030FD90E81C
:10173000922B23E02093E9002091EB0020FF34C09E
:101740002091EE0027FF30C020912F09222321F0A5
:101750002091E80025FF28C010922F0926E0309143
:10176000E80035FF14C08093F1008091E80085FD0A
:1017700027C08091E80080FFFCCF8091E8008E7741
:101780008093E8009F709093E90080E00895309185
:101790003F09343049F43091EB0035FD05C021504C
:1017A00041F481E080932F099F709093E9008FEFBF
:1017B0000895EFE9FFE03197F1F700C00000CFCFC7
:1017C0008FB7F89421E0209330098FBFDBCF80934F
:1017D0002C0970932E0960932D0980913F09843064
:1017E00001F582E08093E9008FEF9091E80081504D
:1017F00095FD06C095ED9A95F1F700008111F5CFA2
:101800008091E80085FF0DC050E040E063E070E0AB
:101810008CE299E00E94B1058091E8008E77809378
:10182000E8000895BC0184E00C94E70BBC0183E060
:101830000C94E70BCF93DF93EC0181E08093E900F8
:101840008FEF9091E800815095FD06C095ED9A9537
:10185000F1F700008111F5CF8091E80085FF14C0F9
:1018600050E040E068E070E0CE010E94B105809158
:10187000E8008E778093E80088E0FE01A5E3B9E0F8
:1018800001900D928A95E1F7DF91CF91089581E063
:101890008093E00080E28093D8001092C9008FE12D
:1018A0009EE40197F1F700C0000087E090EBDC01B7
:1018B0008093A9099093AA09A093AB09B093AC09AE
:1018C00088E19CE00FB6F894A895809360000FBE65
:1018D00090936000FFCF8554990BBC01990F880B42
:1018E000990B0E94A42E20E030E040E451E40E94D5
:1018F000FA2D9B01AC0160E070E080E090E40E9472
:10190000233020E030E04CED53E40E94B62F0895E0
:10191000CF92DF92EF92FF920F931F93E091A50970
:10192000EE2309F414C2E15088E0E802F00111242A
:10193000EB59F64FC280D380E480F58020E030E0A0
:10194000A901C701B6010E94F52D18160CF0FFC1C0
:1019500080916309909164090E94F0068C0164E60D
:1019600070E00E944C2CE0916209E93038F4F0E01C
:10197000E456FE4C0C94742C10926109809160091D
:10198000882371F10E94FF06BC0190E080E00E9474
:10199000A22E20E030E048E451E40E94FA2D20E03D
:1019A00030E040EA51E40E94EA2E0E946C2E660F5D
:1019B000771F660F771F695F7A4FFB016081718126
:1019C0008281938120E030E040E05FE30E94233099
:1019D0009B01AC01C701B6010E94B62F6B017C01CF
:1019E000C701B6011F910F91FF90EF90DF90CF904C
:1019F00008951092610981E080936009BFCF109231
:101A000061096431710538F46A30710540F089E18B
:101A100080939204B3CF88E1693C7105C8F38CE0F0
:101A2000F7CF1092610920E030E040EA52E4C701AC
:101A3000B6010E94F52D87FDA1CF20E030E040E205
:101A400053E4C701B6010E94F52D87FF28C00E940C
:101A5000C62C68E270E00E94602CBC01645C7F4F81
:101A6000072E000C880B990B0E94A42E6B017C01A1
:101A70000B30110508F498C00531110508F0B1C00C
:101A80002EEC2003C001219F900D1124865E9B4FF8
:101A90006AE070E00E944C2C609392046FCF20E0CB
:101AA00030E040EA53E4C701B6010E94F52D87FFFC
:101AB00024C00E94C62C68EE73E00E94602CBC011A
:101AC00068517C4F072E000C880B990B0E94A42EA6
:101AD0006B017C010630110508F466C00531110563
:101AE00008F07FC02EEC2003C001219F900D11242F
:101AF000865E9B4F6FE070E0CDCF20E030E040E2AB
:101B000054E4C701B6010E94F52D87FF23C00E944F
:101B1000C62C60ED77E00E94602CBC016854744FC5
:101B2000072E000C880B990B0E94A42E6B017C01E0
:101B300000311105C8F10531110508F052C02EEC35
:101B40002003C001219F900D1124865E9B4F65E00C
:101B500070E0A0CF20E030E040EA54E4C701B601D5
:101B60000E94F52D87FF0ACF0E94C62C60ED77E01A
:101B70000E94602CBC016854744F072E000C880B27
:101B8000990B0E94A42E6B017C010432110560F0B8
:101B90000333110530F52EEC2003C001219F900D79
:101BA00011248A50964FA6CF82E332CF81E08093F2
:101BB00061096431710590F420E030E040E85EE3B3
:101BC0006A30710520F020E030E040E05FE3C701BB
:101BD000B6010E94B62F6B017C0121CF693C7105D3
:101BE00018F010929204CACE90E080E00E94A22EDB
:101BF00020E030E040EA51E40E94882D20E030E00F
:101C000044E353E40E94FA2D9B01AC010E94B62FDD
:101C100020E030E048E451E40E94B62F0E94732E89
:101C20008CE0861BF5CE81E0809361092AE0269F37
:101C3000C001279F900D112468EB7BE00E944C2C83
:101C40008C5D954097FF03C0919581959109BC01EA
:101C50007727072E000C880B990B0E94A42E2EE3E9
:101C600033EC4EE259E30E94B62F20E030E040EC26
:101C70005EE30E94892D0E94732E0ECF81E0809337
:101C80006109C80183709927892B19F1C8018170F6
:101C9000992724E6289FB001299F700D112490E018
:101CA00080E00E94A22E20E030E040E05EE30E944F
:101CB000B62F20E030E040E45FE30E94892D0E94CF
:101CC000732E6093920407701127012B09F056CEF2
:101CD00088CF82E380939204F6CF81E080936109FC
:101CE00082E3809392040C3F1A4308F447CE90E0BD
:101CF00080E00E94A22E20E030E047E153E40E9401
:101D0000882D20E030E04AE754E40E94FA2D20E0DC
:101D100030E048E452E40E94B62F20E030E040EA90
:101D200051E40E94EA2E0E946C2E660F771F660F08
:101D3000771F695F7A4FFB01208131814281538196
:101D4000C701B6010E94B62F6B017C0117CEC12CD2
:101D5000D12C760145CE682F86E090E00C94F12CD2
:101D6000CF93C0912009C1708091A80980FF29C03C
:101D70001F92CF938EEB97E09F938F930E9458050D
:101D80000F900F900F900F90CC23E9F080912009D5
:101D900080FF3BC0809120098E7F809320090E94A4
:101DA000AB0E8091A80980FF08C089E997E09F9356
:101DB0008F930E9458050F900F9080E0CF910C9464
:101DC0004307C111E7CF8091200980FD1EC08160CB
:101DD00080932009813019F489E080932009809153
:101DE00020090E94AB0E8091A80980FF08C08CEAF0
:101DF00097E09F938F930E9458050F900F908091CA
:101E00002009869586958695D9CFCF9108959F9282
:101E1000AF92BF92CF92DF92EF92FF920F931F93F8
:101E2000CF93DF938C01EB01942E79010E94B00EC9
:101E30002FEF61EE84E0215060408040E1F700C068
:101E400000000E94B00E992DEAEF9E02600111245D
:101E50008091A8098170C017D10739F05E01AC0CE0
:101E6000BD1CF5019281911139C0882341F1CE0149
:101E7000801B910B959587952BEA3AEA829FA001EA
:101E8000839F500D929F500D1124692D6403900182
:101E9000659F300D112481E0981641F182E03F9357
:101EA0002F931F928F9383EE91E09F938F930E94C5
:101EB00058050F900F900F900F900F900F90F70113
:101EC000D183C083DF91CF911F910F91FF90EF904D
:101ED000DF90CF90BF90AF909F900895882321F01E
:101EE0008DE092E00E94BF04E501B2CF81E0D7CF40
:101EF000FF920F931F93CF93DF938C01EB01F42E8E
:101F0000F901A091A609B091A7098281811110C0A1
:101F10000A171B0769F48091A80980FF71C08DE939
:101F200098E0DF91CF911F910F91FF900C94BF0427
:101F30002F2D86E02802A0011124CD01841B950BD2
:101F4000C817D90709F462C086E001900D928A95FE
:101F5000E1F78091A6099091A709840F951F9093AE
:101F6000A7098093A6098091A80980FF49C04F2D39
:101F70000F2C000C550BC01BD10BD595C7956BEAE8
:101F80007AEAC69FC001C79F900DD69F900D11247D
:101F9000849F9001859F300D949F300D11242F5FF9
:101FA0003F4F8091A6099091A709801B910B9595B1
:101FB0008795869FF001879FF00D969FF00D112465
:101FC000E49FB001E59F700DF49F700D112491E026
:101FD00082E0F91201C081E03F932F937F936F93CA
:101FE0001F928F9387E798E09F938F930E945805E5
:101FF0008DB79EB708960FB6F8949EBF0FBE8DBFE3
:10200000DF91CF911F910F91FF9008950E94B00E24
:102010009FEF21EE84E0915020408040E1F700C026
:1020200000000E94B00E9FCFCF9384E090E00E940A
:10203000E32CC82F82E290E00E94E32C982F8C2F93
:10204000CF9108950F931F93CF93DF938091D00882
:102050009091CF08892B80935A059091D1089923AC
:1020600091F0892B80935A0520E08CE595E0FC01E6
:102070003191CF0131112F5FF5E082369F07B9F71B
:1020800021110E944A0A48E050E067EC78E08AE5B6
:1020900095E00E94D62C892B09F445C088E0EAE53A
:1020A000F5E0A7ECB8E001900D928A95E1F7E09198
:1020B0002309F09124093097B1F10280F381E02DDA
:1020C0008AE595E009958091A80982FF2CC080FFE0
:1020D00004C08AE497E00E94BF04D0E0C0E004E4BA
:1020E00017E08091A80980FF0EC0FE01E65AFA4F62
:1020F00080811F928F931F930F930E9458050F901A
:102100000F900F900F902196C830D10551F7809114
:10211000A80980FF08C082E497E0DF91CF911F916A
:102120000F910C94BF04DF91CF911F910F910895EF
:1021300090E080E00E94210790E080E00E940B0781
:102140001092CF080C9422106093490970934A09A9
:1021500080934B0990934C090C9498100F931F9304
:102160006091490970914A0980914B0990914C09FD
:102170008B019C0108711127222733270831110593
:102180002105310529F460641F910F910C94A4106E
:102190006F7BFACF0F931F9341E050E060E070E057
:1021A00004C0440F551F661F771F8A95D2F7CB01D5
:1021B000BA016095709580959095009149091091AC
:1021C0004A0920914B0930914C09602371238223E5
:1021D00093231F910F910C94A4109091C6088095A1
:1021E00089238093C608282F277091F4282F082E62
:1021F000000C330B9217130659F09091E70892FDEB
:1022000007C08595859585950E94CA101092C608CD
:102210000895CF93DF93D82FC091E708C2FB88279A
:1022200080F98D1711F1D0FBC2F9C093E7086091D6
:10223000E60884E090E00E94F12C6C2F82E290E0AE
:102240000E94F12C82E00E94ED108091A80980FF8D
:102250000CC01F92DF938DE297E09F938F930E94B3
:1022600058050F900F900F900F90DF91CF91089528
:102270000F931F9341E050E060E070E004C0440F12
:10228000551F661F771F8A95D2F780914909909153
:102290004A09A0914B09B0914C098A019B01082B76
:1022A000192B2A2B3B2BC901B8011F910F910C94BC
:1022B000A4106093D2087093D3088093D4089093AD
:1022C000D5080C9498101092D008ECE5F5E086E063
:1022D000DF011D928A95E9F70C949810CF93DF9354
:1022E000EC018091A80980FF04C08EEC98E00E9468
:1022F000BF040E94B00E2FEF81EE94E02150804089
:102300009040E1F700C000000E94B00E0E946311EF
:1023100060E070E0CB010E94A410D093A709C093A5
:10232000A609DF91CF9108951F93CF93DF93CDB787
:10233000DEB7AA970FB6F894DEBF0FBECDBF81E41B
:1023400099E02091F100DC012D93CD01B9E08934B1
:102350009B07B9F780914209833009F470C0B8F443
:10236000813009F447C0823009F4B1C08091E8009F
:1023700083FF84C280914109909142099A3008F00C
:102380007DC2E92FF0E0EB55FE4C0C94742C8A30A2
:1023900009F48CC08B3009F46FC0893039F7809113
:1023A0004109813219F780914509909146090297B8
:1023B000E8F68091E800877F8093E8008091E8004C
:1023C00082FF38C09091F3008091F200029731F4BF
:1023D0008091F100813011F0863021F48091F1007C
:1023E000809334098091E8008B778093E8000E9405
:1023F000DB05BCCF80914109813A09F0B7CF8091CC
:10240000E800877F8093E800809145099091460914
:10241000892B61F468E085E399E070E00E948D0605
:102420008091E8008B778093E800A0CF60E090E097
:1024300080E0F3CF80913F098111C0CF97CF809189
:102440004109813A09F092CF80914509909146095E
:10245000892B09F08BCF8091E800877F8093E8007B
:102460008091E80080FFFCCF809191048093F1007F
:102470008091E8008E77B9CF80914109813209F0CF
:1024800075CF8091450990914609892B09F06ECF4F
:102490008091E800877F8093E8000E94DB058091AF
:1024A0004309809391040E94631160CF8091410998
:1024B000813209F05BCF8091E800877F8093E8004C
:1024C0000E94DB0580914409809333094FCF8091AE
:1024D0004109813A09F04ACF8091E800877F8093D3
:1024E000E8008091E80080FFFCCF80913309BECFE7
:1024F000803899F0823809F0C1C1809145098F7008
:10250000873008F0BBC18093E9008091EB0085FB28
:10251000882780F91092E90006C080913D099091CA
:102520003E09911182609091E800977F9093E800B6
:102530008093F1001092F1008091E8008E779AC1AB
:10254000882309F488C1823009F098C18091430939
:1025500081118BC1809145098F702FEF280F263094
:1025600008F08CC18093E9002091EB0020FF7DC131
:10257000933031F48091EB0080628093EB0075C161
:102580009091EB0090619093EB0021E030E001C06E
:10259000220F8A95EAF72093EA001092EA008091D0
:1025A000EB008860EACF811169C1109143091F7760
:1025B0008091E3008078812B8093E3008091E80094
:1025C000877F8093E8000E94DB058091E80080FF10
:1025D000FCCF8091E30080688093E30082E01111DA
:1025E00083E080933F094AC18058823008F046C199
:1025F00020914309309144092C3DE3E03E07A1F5C9
:1026000083E08A838AE289834FB7F894DE011396C8
:1026100020E03EE051E2E32FF0E050935700E491D8
:1026200020FF03C0E295EF703F5FEF708E2F90E0C8
:10263000EA30C0F0C7968D939D932F5F243159F7F0
:102640004FBF8091E800877F8093E8006AE270E0E6
:10265000CE0101960E948D068091E8008B778093D1
:10266000E8000CC1C096E7CF8091450990914609DA
:10267000432F55274330510509F44AC078F54130BE
:10268000510509F47AC08BE590E0E8EEF7E04230BE
:10269000510509F0F3C02091E800277F2093E8005E
:1026A00020914709309148098217930708F49C014B
:1026B00040E02115310509F065C0411163C08091EA
:1026C000E80082FDC9CF80913F09882329F2853037
:1026D00019F28091E80083FFF2CFBECF413251055D
:1026E00009F43CC04232510509F0C8C0833091055D
:1026F00008F0C4C0FC01EE0FFF1FE550FB4F019036
:10270000F081E02D88509B4FDC018C9190E01AC045
:10271000332721303105D1F02115310561F0223008
:10272000310509F0ABC0E5E5F8E0E4918E2F90E0CB
:10273000E5E5F8E007C0E3E7F8E0E4918E2F90E0EC
:10274000E3E7F8E0009709F499C0A5CFE7E6F8E0E1
:10275000E4918E2F90E0E7E6F8E0F4CF8330910526
:1027600008F08CC0880F991FFC01EF5FFA4F0190B1
:10277000F081E02D89E090E08ECF82E190E0E3E40B
:10278000F8E089CF80913F09882309F465CF85302F
:1027900009F462CF8091E80083FD5ECF8091E8006C
:1027A00082FD8DCF8091E80080FF83CF9091F30070
:1027B0008091F2002115310519F08830910550F013
:1027C00041E0089709F040E08091E8008E7780931F
:1027D000E8006FCF44914093F100319621503109C8
:1027E0000196E8CF803809F049C08091E800877FE2
:1027F0008093E800809140098093F1009DCE811183
:102800003DC0109143091230C8F58091E800877FE0
:102810008093E800109340090E94DB05112311F01A
:1028200084E005C08091E30087FDFACF81E08093CA
:102830003F0942E061EC81E00E94FA0542E261EC6E
:1028400082E00E94FA0542E261EC83E00E94FA0510
:1028500080913F0913C080914309813079F481E070
:10286000933009F080E080933E091092E900809156
:10287000E800877F8093E8000E94DB058091E800F4
:1028800083FF0AC08091E800877F8093E8008091F1
:10289000EB0080628093EB00AA960FB6F894DEBF3F
:1028A0000FBECDBFDF91CF911F910895882321F0F6
:1028B0000E94500A0C9422100895882339F09091B8
:1028C000D008982B9093D0080C9422100895882358
:1028D00009F44BC0823871F40E94370781FF45C06C
:1028E00089E30E94640A0E94221089E30E94570A29
:1028F0000C942210833859F40E94370780FF35C0AA
:1029000083E50E94640A0E94221083E5EFCF843899
:1029100059F40E94370782FF28C087E40E94640AA6
:102920000E94221087E4E2CF9CEF980F913AF0F2D8
:1029300090E2980F983050F4877091E001C0990FA1
:102940008A95EAF7892F0E94500AD2CF9BE5980F0B
:10295000933020F490E080E00C942107885A87316E
:1029600020F490E080E00C940B0708956F927F9222
:102970008F929F92AF92BF92CF92DF92EF92FF928F
:102980000F931F93CF93DF93CDB7DEB72A970FB680
:10299000F894DEBF0FBECDBF8E010F5F1F4F8AE0E0
:1029A000F80111928A95E9F797EEE92E94E0F92E55
:1029B00068012CEE622E24E0722E88248394912CE0
:1029C000F70181917F018F3F09F446C0F894E82F09
:1029D000E295EF70F0E021A18F70A40102C0440FD6
:1029E000551F8A95E2F7CA01922F982B91A392A1C5
:1029F0008095892382A3789400C0ECEEF4E021E076
:102A000030E0B12CA12C41914F3F09F47FC0A42F9D
:102A1000A295AF70B0E090968C9190E04F7002C09C
:102A2000959587954A95E2F780FD70C0C901A82A5F
:102A3000B92A220F331F54E0E83FF50721F7F701C9
:102A4000319780818F3F11F00E94730880EA8A9548
:102A5000F1F7F601B182A082F2E0CF0ED11C6E1424
:102A60007F0409F0ADCF4AE050E0B8018CED98E06A
:102A70000E94D62CFF24F394009709F4F12C892BA3
:102A800009F447C08AE0F801ACEDB8E001900D927E
:102A90008A95E1F781E08093D8080E94FF06909321
:102AA000D7088093D6088091D6089091D7080E94C5
:102AB000F006059790F18091DC089091DD089093E5
:102AC000E9088093E8088091DE089091DF089093F0
:102AD000EB088093EA088091E0089091E1089093D8
:102AE000ED088093EC088091E2089091E3089093C0
:102AF000EF088093EE088091E4089091E5089093A8
:102B0000F1088093F0081092D80807C090E080E0A8
:102B10008ECF8091D8088111C6CF8091DB088823A1
:102B200089F08091D9089091DA080E94F006893ED8
:102B3000934040F083EE0E94671482EE0E94671477
:102B40001092DB088F2D2A960FB6F894DEBF0FBEC9
:102B5000CDBFDF91CF911F910F91FF90EF90DF904C
:102B6000CF90BF90AF909F908F907F906F9008957F
:102B7000CF93C82F882309F488C08238C1F40E94FB
:102B8000370781FD82C089E30E94640A0E942210F7
:102B90002FEF81EE94E0215080409040E1F700C09B
:102BA000000089E30E94570ACF910C9422108338C9
:102BB000A1F40E94370780FD68C083E50E94640A83
:102BC0000E9422102FEF81EE94E02150804090402F
:102BD000E1F700C0000083E5E5CF8438A1F40E944E
:102BE000370782FD52C087E40E94640A0E942210C7
:102BF0002FEF81EE94E0215080409040E1F700C03B
:102C0000000087E4CFCF8CEF8C0F813A68F4ECE5BD
:102C1000F5E08191C81799F125E0E236F207C9F78E
:102C20008C2F0E94640AC0CF80E28C0F883068F439
:102C3000C77021E030E001C0220FCA95EAF7809109
:102C4000D008822B8093D008AFCFEBE5EC0FE330B8
:102C500040F4F0E0EA54FB4F808190E0CF910C9477
:102C60002107C85AC73188F4EC2FF0E0EE0FFF1FA0
:102C7000E754FB4F80819181CF910C940B078C2FEF
:102C80000E94570A0E942210CBCFCF9108951F9324
:102C9000CF93DF93182FD0E0C0E0893311F4C0E563
:102CA000D0E0812F0E94B815209731F4812FDF9159
:102CB000CF911F910C9467148FE99FE00197F1F772
:102CC00000C000002197F0CF0F931F93CF93DF93A5
:102CD000C62FD42F022FFC0182818823A1F060939C
:102CE0004F090E94FF0690934E0980934D09C770CB
:102CF00081E001C0880FCA95EAF7DF91CF911F915B
:102D00000F910C945D1480914F09681335C0809128
:102D10004D0990914E090E94F006883C910560F59E
:102D200010E21D0FCD17B9F080E28C0F883040F40F
:102D3000C77081E001C0880FCA95EAF70E94561457
:102D4000183048F481E09D2F977001C0880F9A9544
:102D5000EAF70E945D14802F0E944716183098F4FD
:102D6000D77081E001C0880FDA95EAF7DF91CF9143
:102D70001F910F910C945614C77081E001C0880F09
:102D8000CA95EAF7F3CFDF91CF911F910F91089584
:102D9000AF92BF92CF92DF92EF92FF920F931F9369
:102DA000CF93DF93EC018AE0A82EFE012491222329
:102DB00009F494C0213009F03EC0319684918130ED
:102DC00031F42296FE0184910E94471607C082309A
:102DD00039F42296FE0184910E94B8152196E5CF20
:102DE000833031F42296FE0184910E946714F6CF5D
:102DF000843009F071C02296FE01249190E080E0B9
:102E0000FE0131962053330B2A30310548F00197EB
:102E100028F3EFE9FFE03197F1F700C00000F7CFAA
:102E2000A89EA001A99E500D1124C901840F951FD1
:102E30002491EF01E5CFE22FF0E0EF58FD4FB49081
:102E4000822F86958695869590E0FC01EF59FD4F7F
:102E5000E4902770F12C022E02C0F594E7940A94B6
:102E6000E2F731E0E322FF24FC01EF5AFD4FC4906A
:102E7000D12C022E02C0D594C7940A94E2F7E1E067
:102E8000CE22DD24FC01EF5BFD4F049110E002C077
:102E9000159507952A95E2F701701127E114F104C1
:102EA00019F081EE0E94B815C114D10419F086EE14
:102EB0000E94B8158B2D0E944716CD2819F086EE7A
:102EC0000E946714EF2819F081EE0E946714012B0D
:102ED00009F484CF8CE278CFEF0180CFDF91CF91DE
:102EE0001F910F91FF90EF90DF90CF90BF90AF9028
:102EF000089569EE7EEF90E080E00E940F2D60E083
:102F000082E090E00E94F12C60E083E090E00E947B
:102F1000F12C1092D2081092D3081092D40810927B
:102F2000D50860E084E090E00E94F12C60E082E24D
:102F300090E00E94F12C60E085E090E00E94F12C8E
:102F400060E086E090E00E94F12C6FEF87E090E077
:102F50000E94F12C40E050E0BA0188E090E00E942D
:102F6000032D60E08DE090E00E94F12C40E050E005
:102F7000BA0188E190E00E94032D60E087E190E0D3
:102F80000E94F12C40E050E0BA018CE190E00E94F8
:102F9000032D70E060E080E290E00E940F2D40E0A1
:102FA00050E0BA0188E190E00E94032D40E050E03B
:102FB000BA018FE090E00E94032D40E050E0BA019A
:102FC00083E190E00C94032D90E080E00E94EB2CD4
:102FD000893E9E4F51F00E9479178091200984709C
:102FE0008961809320090E94AB0E86E090E00E94E8
:102FF000E32C80932009803220F0877088618093D1
:10300000200990912009892F817090FF04C0892F99
:103010008695869586950C94430780915E0981116B
:1030200034C090E080E00E94EB2C893E9E4F11F06E
:103030000E94791787E090E00E94E32C80935F095B
:10304000E5E6F9E080E090E0A0E8BFEB11821082B5
:1030500082839383A483B58317821682389629E0EE
:10306000E53AF20799F780915E0981110CC00E9440
:10307000E7073E9A82E0809390008AE18093910076
:1030800081E080935E090C94460808957F928F92A8
:103090009F92AF92BF92CF92DF92EF92FF920F93E7
:1030A0001F93CF93DF934B015C017A0180915F09FD
:1030B00080FF85C080915E09811102C00E940D18B9
:1030C00020E030E0A901C501B4010E94F52D87FF81
:1030D00004C0B7FAB094B7F8B0947090A509872DE2
:1030E0008150990B6C01EC01CF3FDC0709F051C016
:1030F00081E0870D893008F489C088E08093A509B4
:1031000085E699E028E0FC013896DC0101900D92FB
:103110002A95E1F7089629E08D39920799F781E021
:103120008093150980935D09C091A509C150DD0BFD
:103130000E94FF06FE0123E0EE0FFF1F2A95E1F734
:10314000EB59F64F9183808382829382A482B58269
:10315000F782E6820E94FF069093640980936309D8
:103160008091D003882359F180917100826080930F
:1031700071008091900080688093900080915D093B
:10318000882321F00E94880C0E94F2071092D0033D
:1031900016C08E0133E0000F111F3A95E1F70B596D
:1031A000164FA5019401F801628173818481958194
:1031B0000E94F52D811128C0CC15DD0574F0DF913A
:1031C000CF911F910F91FF90EF90DF90CF90BF9024
:1031D000AF909F908F907F900895219688E0F8019E
:1031E0003896D80101900D928A95E1F70E94FF066A
:1031F000F8019187808782869386A486B586F786B4
:10320000E686085F1F4FD8CF21976ECF8093A50920
:1032100086CFCF92DF92EF92FF92CF93DF93EC01B4
:103220007B0180915F0980FD08C0DF91CF91FF9005
:10323000EF90DF90CF900C94460880915E09811149
:1032400002C00E940D1880915D0981110E944608FC
:1032500081E080935C0910925B09D0935A09C09376
:103260005909F0925809E0925709109256091092A4
:103270005509109254096C817D818E819F810E9435
:10328000732E9B01A0E6BAEE0E94792DC12C2EE18F
:10329000D22EE12CF12CA70196010E94572D6881B6
:1032A00079818A819B81A9010E9446180E94FF06AC
:1032B0009093530980935209E0915909F0915A096A
:1032C000809154099091550933E0880F991F3A95E0
:1032D000E1F7E80FF91F64817581868197810E946B
:1032E000732E9B01A0E6BAEE0E94792DA7019601EC
:1032F0000E94572D3093510920935009DF91CF91AF
:10330000FF90EF90DF90CF90089581E080931F09A8
:1033100068E070E081E594E00C9409190E946D0862
:1033200010921E0968E070E081E194E00C940919A4
:1033300081E080931E0968E070E081ED93E00C94D9
:10334000091962E070E080EC93E00E9409192FEF08
:1033500081EE94E0215080409040E1F700C00000F1
:103360000E94460860915F096E7F60935F0987E065
:1033700090E00C94F12C60915F09616060935F09AB
:1033800087E090E00E94F12C62E070E080EB93E037
:103390000C940919CF92DF92EF92FF92CF93C82F2E
:1033A00020E8829FC001112460E170E08C5F9E4F95
:1033B0000E940919C12CD12C7601C39404C0CC0CF5
:1033C000DD1CEE1CFF1CCA95D2F76C2D83E090E04B
:1033D0000E94F12CC701B601CF91FF90EF90DF90D2
:1033E000CF900C9459110E946B0C4FEF5FEF0C942F
:1033F0004618CF92DF92EF92FF920F931F93CF93D5
:10340000DF936B017C0120E030E0A9010E94F52DE3
:1034100087FF04C0F7FAF094F7F8F09480915D0903
:10342000882309F458C080915E09811102C00E946E
:103430000D1805E619E0C7E0D0E0A7019601F801F4
:1034400062AD73AD84AD95AD0E94F52D81113CC088
:1034500083E0CC0FDD1F8A95E1F7CB59D64F198257
:10346000188280E090E0A0E8BFEB8A839B83AC8366
:10347000BD831F821E82AC01BD01F9E0CD39DF079B
:1034800089F4C1E0C09315098091A509815080930A
:10349000A509811120C00E94E707C093D0031092B4
:1034A0005D0919C088E0FE013896DE0101900D9299
:1034B0008A95E1F7198618864A875B876C877D872E
:1034C0001F861E862896D9CF219708501109CF3F15
:1034D000DC0709F0B2CFDF91CF911F910F91FF90E0
:1034E000EF90DF90CF9008954F925F926F927F920E
:1034F0008F929F92AF92BF92CF92DF92EF92FF9204
:103500000F931F93CF93DF93CDB7DEB7A8970FB676
:10351000F894DEBF0FBECDBF7C01DC0113968D9108
:103520009C911497892B49F01C911196DC90812F66
:103530008D218F3F11F00C943B23A8960FB6F89481
:10354000DEBF0FBECDBFDF91CF911F910F91FF90D6
:10355000EF90DF90CF90BF90AF909F908F907F9033
:103560006F905F904F9008950E94870A082F682FF0
:1035700089819A810E94210BE12FF0E0BCE0DB9E63
:10358000E00DF11D11242CE3029FE00DF11D11242B
:10359000EE0FFF1FEB51FC4F0591149180916208D3
:1035A00081116DC0D70112968C9181110AC005302E
:1035B000BDE51B0709F453C090F40430FDE51F0777
:1035C000F9F0D70112968C91F801E75AFD45ED30DC
:1035D000F10508F051C1E155FE4C0C94742C0730F4
:1035E0002DE5120709F441C008303DE5130749F7FE
:1035F00060910402709105024FEF8CE598E03CC0A9
:1036000082E695E00E946E1181E0809362088091CD
:10361000C608877009F491CFD70112968C91882340
:1036200009F48BCF8091E70882FD87CF82E0A896CE
:103630000FB6F894DEBF0FBECDBFDF91CF911F91C3
:103640000F91FF90EF90DF90CF90BF90AF909F9041
:103650008F907F906F905F904F900C94ED108CE561
:1036600098E00E946E1182E0D0CF609106027091C6
:10367000070241E082E695E00E94DD25C8CF0630D2
:103680009DE5190799F020F00930BDE51B0780F191
:103690008130B9F1823009F094CF609106027091C7
:1036A000070297014FEF8CE598E033C0F701928154
:1036B000992309F4ACCF813029F0823079F010924F
:1036C0006208A5CF6091A6097091A70926E032E0B3
:1036D00041E082E695E00E94070FF1CF6091A609D4
:1036E0007091A70924E032E04FEF8CE598E0F3CF2A
:1036F0008091A80980FF8BCF81EF92E00E94BF04E8
:1037000086CF6091040270910502970141E082E644
:1037100095E00E94780F55CF882309F478CF80E098
:103720000E94CA1974CF882309F471CF81E0F8CFC1
:10373000882321F082E00E94381169CF82E00E9444
:10374000CA1065CF882311F085E0F5CF85E0F7CF6B
:10375000882331F083E00E9438110E94AE1057CFC9
:1037600083E00E94CA10F9CF882311F084E0F3CFE0
:1037700084E0F7CF882321F08AE693E00E94C81600
:10378000F70182810F31FCE51F0709F489C0D701D9
:1037900012968C910A32BCE51B0709F088C0882379
:1037A00009F492C08091620990E0019669E070E0AE
:1037B0000E94602C8093620964E070E089E092E0EE
:1037C0000E94091924CF8823D9F28BE493E0D6CF45
:1037D0008823B1F28DE393E0D1CF882389F28AE286
:1037E00093E0CCCF8823D1F08091DB0881110AC00F
:1037F00081E08093DB088091080281110DC082EE88
:103800000E94B8150E94FF069093DA088093D908A9
:103810008BE20E94B815B4CF83EEF2CF8BE20E9408
:103820006714AECF90910802882361F0911102C015
:1038300086E4EFCF81EE0E94B81583EE0E94B815A2
:1038400081E2E7CF911102C086E4E9CF81EE0E94C8
:10385000671483EE0E94671481E2E1CF882309F4A4
:103860008FCF80910802811104C081E0809308020B
:1038700087CF1092080284CF0D31BCE51B0731F4CD
:10388000882309F484CF0E94BB19C1CE0E31ECE528
:103890001E0709F075CF882351F00E94A119B7CEF9
:1038A000882391F080915F0980FDF7CFECCFF7017D
:1038B00082810B32FCE51F0739F4882329F08091BF
:1038C000620990E0089672CFD70112968C918823F6
:1038D00009F4F2C60E3BBCE51B0709F474C0D0F432
:1038E0000C3BFCE51F0709F44EC00D3B2CE512070D
:1038F00009F461C006329CE5190709F4CBC0073210
:10390000BCE51B0709F0BBC0882309F4DAC60E9496
:103910008E197DCE003C3CE5130709F4AAC008F4DB
:1039200083C0013CACE51A0729F790912009892F43
:103930008695869586958F5F8F719770843008F095
:103940009BC0880F880F880F892B80932009809156
:103950002009887F91E009F490E08091200990FB94
:1039600080F9809320090E94AB0E8091A80980FF06
:1039700053C0809120098695869586951F928F93D6
:103980008EEA93E041C0809120098770886180931E
:103990002009887F91E009F490E08091200990FB54
:1039A00080F98093200983E00E94430780912009D9
:1039B0000E94AB0E2CCE8091200987708E7F809361
:1039C000200980E0F1CF80912009982F987F79F02D
:1039D000885080932009887F91E009F490E08091DD
:1039E000200990FB80F9809320090E94AB0E809102
:1039F000A80980FF11C0809120098695869586953B
:103A00001F928F938EE793E09F938F930E945805A8
:103A10000F900F900F900F908091200986958695BA
:103A200086950E944307F3CD80912009982F9695A3
:103A300096959695933040F49F5F990F990F990F43
:103A40008770892B80932009809120098160809361
:103A500020090E94AB0E8091A80980FFDDCF8091E4
:103A600020098695869586951F928F9386E993E027
:103A7000CBCF0E94B00ECBCD9093200968CF0832F7
:103A8000ECE51E0751F490911E09882309F419C62C
:103A900091113DCF0E949819BACD0C32FCE51F0759
:103AA00031F4882309F40DC60E948519B0CD0D327A
:103AB0002CE5120751F4882309F403C610921F095C
:103AC00068E070E089E292E07BCE0E323CE51307BD
:103AD00041F4882309F4F5C580911F098111EECFC7
:103AE000E3CF09329CE5190709F0EBC5882309F4F7
:103AF000E8C50E946D082091090330E02F5F3F4F19
:103B0000237033272093090348E2429FC001439F5B
:103B1000900D112465E070E087599D4F51CE023E13
:103B2000110571F40E946D0880916408882319F0D2
:103B300081E080936308109264081092100967CDA9
:103B4000033E110591F490916308992321F10E949D
:103B50006D081092640881E08093100910920D099D
:103B600010920F0910920E0952CD0235110551F431
:103B70008091AE039091AF030A979093AF03809327
:103B8000AE0345CD0135110531F48091AE0390911E
:103B9000AF030A96F2CF9091090391117AC0D70131
:103BA00011969C91119725E030E0291B3109DC909A
:103BB000B0E1DB0EECE02E9FD00C1124882309F439
:103BC000ABC0442319F08D2D0E94F3198091640835
:103BD000882351F080910C09E82FF0E0E450F74F72
:103BE000D0828F5F80930C090115110509F00FCD6C
:103BF000D70112968C91882309F452C510924F096F
:103C00000430BDE51B0708F0CAC00B3FECE51E07FA
:103C100038F4980122503C452431310508F0C9C0E0
:103C20000E9414109093E7088093E60801313CE568
:103C3000130709F4A4C108F008C109309CE519076D
:103C400009F471C108F0DDC00530BCE51B0709F4BB
:103C50005EC108F0C6C00330FCE51F0709F44DC182
:103C600008F051C18091E608816002301C4509F4DA
:103C700047C16091E6081091E70884E090E00E9457
:103C8000F12C612F82E290E00E94F12C0E946311DE
:103C9000BECC913081F4D70111969C91119725E00B
:103CA00030E0291B3109D22EDD0CDD0CD20E9C91A7
:103CB0009D5CD90E83CF923071F4F701918125E09C
:103CC00030E0291B3109D080F3E3DF0E97E0299F14
:103CD000D00C112473CF6CE0D62E933009F06ECF48
:103CE00093E2E3E9F4E0DE01119601900D929A95DA
:103CF000E1F7D701EC91EC0FFD2FF11D11969C918E
:103D000025E030E0291B3109D084BCE02B9FD00C8A
:103D10001124E9E0DE0E52CF442309F465CF8D2D46
:103D20000E946B0C0E94F9195FCF043FFCE51F074E
:103D300039F188F4093D3CE51307F1F00A3D8CE5C3
:103D4000180751F1083D9CE5190709F051CF26E20B
:103D500041EE61EE0DC0063FACE51A07C9F0A0F0D8
:103D600027E245EE66EE073FECE51E0709F040CF7F
:103D7000C7010E9464164BCC27E245EE65EEF8CFF2
:103D800026E241EE60EEF4CF27E245EE64EEF0CF9E
:103D900026E241EE62EEECCF28E241E0EFCF0236C0
:103DA000FDE51F0709F43CCF063A2DE5120709F49B
:103DB00037CF06313CE5130709F027C1882309F402
:103DC00073C48091D0088A7A91E009F490E09093CE
:103DD0006508811116C189E20E94640A0E942210BE
:103DE00016CC07308CE5180709F499C08091E608D5
:103DF000806108301C4508F483C08091E608806427
:103E00007FC00D30ACE51A0709F4ADC058F40B3093
:103E1000ECE51E0709F4A3C008F48BC08091E60806
:103E20008D7F6EC08091E6088F7E0F302CE51207E3
:103E300009F466C08091E608877F00311C4508F4CC
:103E40005FC08091E6088F7D5BC00E3F8CE5180750
:103E500009F491C038F50531ACE51A0709F4ADC095
:103E600080F40331ECE51E0709F493C008F48BC01D
:103E70000E9463119091E608892F97FB87F980587B
